:020000000140BD
:020003000157A3
:05000B0002005101405C
:2000400075811AD2AFD2A9D28C12005A12001B80FB438CDC050832050832740075F000F52B
:200060000985F00A740075F000F51585F016748075F025C0E0C0F0120C0015811581120C54
:200080004F79307A0EE98AF0C0E0C0F0120C23158115811201F312018B1202061208951241
:2000A00002561203751204811206471205EB1206F61208B51209A2020096227F09120CDE8E
:2000C000740078FC120CD2F6740075F00008F608A6F078FC120CD2E6120D047B0A120CFBD2
:2000E000120DD145F0700302013D801678FD120CD2E60886F0120D8E18F608A6F0120D97BA
:2001000080D0741175F000C0E0C0F0120C3715811581120C4FC0E0C0F0120C5F158115816E
:2001200078FC120CD2F608E60886F079F6120CD7120CF478FC120CD2E6F70200EC78FD12CD
:200140000CD2E60886F079F6120CD7120CF47400F778FD120CD2E60886F07B007C00120D9D
:20016000C845F0700302017074FF75F0FF02018679F6120CD7E98AF0C0E0C0F0120C7F1573
:200180008115810201867FF7020CEDE598540175F0007B007C00120DD145F070030201B3D2
:2001A000120C4FC0E0C0F0120C5F15811581F5100201B774FFF51022E598540175F0007BCE
:2001C000007C00120DD145F070030201D5120C74F5100201D974FFF5102212024379637A79
:2001E0000EE98AF0C0E0C0F0120C23158115811201F322795F7A0EE98AF0C0E0C0F0120C78
:20020000231581158122E510120D047B0A120CFB120DC845F0700302022F79307A0EE98A51
:20022000F0C0E0C0F0120C23158115811201F322C292746475F000C0E0C0F0120CB515819F
:20024000158122D292746475F000C0E0C0F0120CB51581158122E510120D047B65120CFBC3
:20026000120DC845F07003020353120230D2B3D2B4C2B5D2B2C2B6C2B7120A19C2B37464DA
:2002800075F000C0E0C0F0120CB515811581E50E75F0007B557C00120DC845F07003020372
:2002A0001AC295746475F000C0E0C0F0120CB515811581C2A700D2A7749675F000C0E0C090
:2002C000F0120CB515811581D292746475F000C0E0C0F0120CB515811581C292746475F0AE
:2002E00000C0E0C0F0120CB515811581C2A700D2A7749675F000C0E0C0F0120CB515811590
:2003000081D292746475F000C0E0C0F0120CB515811581C292D29502032EC2A7740A75F032
:2003200000C0E0C0F0120CB515811581D2A7740A75F000C0E0C0F0120CB515811581D2B33E
:20034000746475F000C0E0C0F0120CB5158115811201DA22851180D29700000000C297002A
:20036000000000E5124480F5A0C2B574FFF580E58075F00022E510120D047B77120CFB12AD
:200380000DC845F07003020480120230D295C297D2B3C2B4D2B5D2B2D2B6D2B7D2A7120AAA
:2003A00019C2B3746475F000C0E0C0F0120CB515811581740075F000F51385F014740075D0
:2003C000F000F50985F00AE509850AF0AB15AC16120DDB45F0700302046B8012E509850A9F
:2003E000F0120D8EF50985F00A120D9780D9741175F000C0E0C0F0120C3715811581E5092B
:20040000850AF0F51185F012851180D29700000000C29700000000E5124480F5A0120A1973
:20042000120C74F580741375F000C0E0C0F0120C3715811581E5138514F02580C5F03400E9
:20044000C5F0F51385F0141209EEE50E75F0007B557C00120DC845F070030204633096FDEE
:20046000020468D2A630A6FD0203DCD2B3746475F000C0E0C0F0120CB5158115811201DAE4
:200480002205810581E510120D047B72120CFB120DC845F07003020539740075F000F51360
:2004A00085F014120230D295C297D2B3D2A7C2B4D2B5C2B2D2B6D2B77431F50D740075F0AF
:2004C0000078FD120CD2F608A6F078FD120CD2E60886F0AB15AC16120DDB45F0700302052F
:2004E00036801678FD120CD2E60886F0120D8E18F608A6F0120D9780D178FD120CD2E608B4
:2005000086F0F51185F012120354F50CE5138514F0250CC5F03400C5F0F51385F014E50C9C
:2005200075F000C0E0C0F012053E15811581D2B51205650204E31201DA158115812278FBEB
:20054000120CD2E6F50BE50B75F0007B047C00120D7DF50B12058878FB120CD2E6540FF599
:200560000B120588221201B87B137C00120DC845F070030205871201B87B117C00120DD1FA
:2005800045F0600302057622E50B75F0007B097C00120DEB45F070030205B0E50B243775A6
:2005A000F000C0E0C0F0120C37158115810205C2E50B243075F000C0E0C0F0120C371581CD
:2005C000158122E58075F0007BFF7C00120DD145F070030205EA7430F50DE519851AF012D5
:2005E0000D8EF51985F01A120D9722E510120D047B62120CFB120DC845F0700302064612EE
:200600000230D2B4D2B5C2B2D2B6C2B774FFF580E580F50CE50C541CF50C746875F00EC067
:20062000E0C0F0E50C75F0007B027C00120D7DC0E0C0F0740275F000120AAB15811581150C
:200640008115811201DA22E510120D047B6C120CFB120DC845F070030206F5120230C2B317
:20066000E50E75F0007B557C00120DC845F07003020675C295D2A7D2B4D2B5D2B2D2B6D20F
:20068000B7746475F000C0E0C0F0120CB515811581120A11740575F000C0E0C0F0120CB5E9
:2006A00015811581C2B6C2B7120A19120A11740575F000C0E0C0F0120CB515811581C2B517
:2006C000D2B6C2B7120A19120A11740575F000C0E0C0F0120CB515811581D292746475F0E9
:2006E00000C0E0C0F0120CB515811581C292D295D2B51201DA22E510120D047B63120CFB4B
:20070000120DC845F0700302073A748075F00EC0E0C0F0E5138514F0120DA12401C5F03401
:2007200000C5F0C0E0C0F0740275F000120AAB15811581158115811201DA22120230C2970E
:20074000D295D2B3D2A7C2B4D2B5C2B2C2B6C2B7743175F000F51185F012120354F50E12BD
:200760000A19E50E75F0007BFF7C00120DC845F07003020784740075F001F51185F0121273
:200780000354F50E74FFF50FD2B52212073BE50E75F0009007F4020D0D740075F010F51797
:2007A00085F018020814740075F010F51785F018020814740075F020F51785F0180208143E
:2007C000740075F020F51785F018020814740075F050F51785F018020814740075F050F56B
:2007E0001785F018020814740075F000F51785F018020814E707FF00DA076500CD0755004B
:20080000C0076200B3075200A60761009907510000001408740075F000F51385F0147400AA
:2008200075F000F51985F01AD2B3D2A7C2B4D2B5C2B2D2B6D2B77431F50D740075F000F5C1
:200840000985F00AE509850AF0AB17AC18120DDB45F070030208948012E509850AF0120DBF
:200860008EF50985F00A120D9780D9E509850AF0F51185F012120354F50CE5138514F02554
:200880000CC5F03400C5F0F51385F0141205C3D2B502085922E510120D047B73120CFB1206
:2008A0000DC845F070030208B41200BBF51585F0161201DA22E510120D047B67120CFB1267
:2008C0000DC845F070030209A112078BE50E75F0007BFF7C00120DD145F0700302098E7458
:2008E0009075F00EC0E0C0F0E50E75F000C0E0C0F0740275F000120AAB1581158115811584
:2009000081E50F75F0007BFF7C00120DC845F07003020924749F75F00EC0E0C0F0120C2332
:2009200015811581E50F75F0007B057C00120DC845F0700302094774A475F00EC0E0C0F07A
:20094000120C231581158174A875F00EC0E0C0F0E519851AF0C0E0C0F0740275F000120A77
:20096000AB158115811581158174BC75F00EC0E0C0F0E5158516F0C0E0C0F0740275F000D1
:20098000120AAB158115811581158102099E74CF75F00EC0E0C0F0120C2315811581120109
:2009A000DA22E510120D047B70120CFB120DC845F070030209ED12078B74E175F00EC0E08C
:2009C000C0F0E50E75F000C0E0C0F0E519851AF0C0E0C0F0E5158516F0C0E0C0F074047520
:2009E000F000120AAB7FF8120CDE1201DA22E50E75F0007B557C00120DC845F07003020A7F
:200A000009C2A700D2A7020A10C2A7000000D2A722C2A7120A62D2A7220581058174007554
:200A2000F00078FD120CD2F608A6F078FD120CD2E60886F07B017C00120DA845F07003029B
:200A40000A5D801678FD120CD2E60886F0120D8E18F608A6F0120D9780D1020A4415811575
:200A6000812205810581740075F00078FD120CD2F608A6F078FD120CD2E60886F07B147C21
:200A800000120DA845F07003020AA6801678FD120CD2E60886F0120D8E18F608A6F0120D5E
:200AA0009780D1020A8D158115812223F42581F8868208868308E4FEFF93700122B425555C
:200AC000A3E493B42D06430780A3E493B4300343074024D0B40A00500CCE75F00AA42EFEA5
:200AE000A3E49380EDE493B46413E60886F030F708430720120D9EA6F018F68003B47505BE
:200B000043070A801CB478054307108014B46F0B430708800C120C3DA3809BB462624307DF
:200B2000027A00C004C005C006C007AB0753031F7C00E60886F0120D4AA6F018F6EDD0074B
:200B4000D006D005D0042430B43A0040022407C0E00AE645F070CCA902EF30E506742D12FE
:200B60000C3D0A120BE1D0E0120C3DD9F90808EF30E7A5EAC39E50A07420120C3D0A80F3E5
:200B8000B4630BAA01120BE1E6120C3D80DFB4732BC082C08386820886837A00E4936004A5
:200BA000A30A80F88683188682120BE1E493A36005120C3D80F6D083D08280B1B469198607
:200BC000017A00E76004090A80F9120BE18601E7609B120C3D0980F7F97A01120BE1E980A6
:200BE000A8EE601B8FF020F716C002EAC39E500D742030F6027430120C3D0A80EED00222A7
:200C000078FB120CD28603088604748075F070120D4A120D9E758921F58DF58B758859757B
:200C200098522278FB120CD28682088683E493602D120C3DA380F678FB120CD2E63099FDA5
:200C4000C299F599B40A17740D80F2E430980C3098FDC298E599B40D02740A75F00022784E
:200C6000FB120CD2E63099FDC299F5992274FFF5F030980A3098FDC298E59975F00022780C
:200C8000FB120CD28601E4FBFCFFE709B42D030FE709C39430B40A005012FA740A75F000B1
:200CA000120D362AFBE5F03400FC80E4EB8CF0DF03020D9E2278FB120CD28603088604BB00
:200CC0000004BC00012279E5A3D9FD1BBBFFF01C80F4C82581C822C92581C97A0022D08386
:200CE000D082CF2581F581CFC082C08322CF2581F581CF2229F9E5F03AFA227C00CB30E7BA
:200D0000011CCB2275F00030E70215F022FDE493A3FEE493A3FF4E7009E493FE740193FFB3
:200D2000800BE493A3B5050BE493B5F0068F838E82E473A380D8FEEBA4FD8EF0ECA4FCEB34
:200D40008EF0A4C5F02C2DC5F022C002C001AAF0F97E007D007F11C3E933F9EA33FADF0815
:200D6000F5F0E9D001D00222ED33FDEE33FEC3ED9BF5F0EE9C40E0ADF0FED380DBBB000145
:200D800022C3C5F013C5F013DBF722120D8E04700205F022120D9714B4FF0215F022120DEB
:200DA00097F4C5F0F4C5F022120DFB4029801E120DFB40227017801E120DFB4010701780F5
:200DC0000C120DFB50108005120E0F6009E4F5F022120E0F60F7E4F5F00422120E0F40F6AB
:200DE00080EB120E0F40EF70E480EB120E0F40DD70E480D9120E0F50DD80D2C39BC5F09C15
:200E000020E70720D207C345F02220D2F9D322C5F0C39C7003E5F09B22FBE493CB22FCE479
:200E200093FB740193CC22FAE493F9740193CA220A20456173792D446F776E6C6F6164654A
:200E4000722056332E3020666F722041544D454C2038394335312F35322F35355744000A11
:200E6000203E000A206F6B000A206C6F636B2062697420312C322C33203D20253033620069
:200E80000A2043484B53554D203D2025303478000A20666F756E6420383943253278002DC9
:200EA000313256002D3556000A206E6F6E626C616E6B202575206279746573000A2062793E
:200EC00074657320636F756E746572202575000A204E6F7420666F756E6420383943787891
:0A0EE0000025782C25752C257500DF
:00000001FF
